:1000000018308A0000280000FF00030E8301A100C1
:100010000A08A0008A010408A2007708A300780853
:10002000A4007908A5007A08A6007B08A70083131E
:1000300083128C308400001C1F280C1841288C303F
:100040008400801E25288C1A3E288C308400801C59
:100050002B288C184428220884002308F700240841
:10006000F8002508F9002608FA002708FB002008F8
:100070008A00210E8300FF0E7F0E09008A110A12EA
:1000800081298A110A124E298A110A1253290A104B
:100090008A100A11820728340C34013406340A10FD
:1000A0008A100A118207203400340A108A100A11BB
:1000B000820741345A3400340A108A100A11820728
:1000C000203445344C3400340A108A100A11820757
:1000D00052346534713400340A108A100A118207D0
:1000E00050346F34733400340A108A100A118207B6
:1000F000533445345434203445344C344534563428
:10010000203454344F3420345A34453452344F342C
:1001100000340A108A100A1182075034753473347F
:100120006834203427345234493447344834543402
:10013000273420347734683465346E3420344F34B7
:100140006B34203400340A108A100A1182074334B9
:100150004F344E34463449344734203445344C34DB
:10016000453456344134543449344F344E342034B9
:10017000543442344C3400340A108A100A11820775
:10018000503475347334683420342734523449344D
:100190004734483454342734203477346834653451
:1001A0006E3420344F346B3400340A108A100A1134
:1001B000820745344C34203454344F3400340A1010
:1001C0008A100A1182072034203449344D345034C7
:1001D0002034203400340A108A100A11F23E031829
:1001E0008A0A820052344534413444342034453440
:1001F0004C342034543442344C3420342F34523470
:10020000693467346834743400340A148A100A116B
:10021000820745344C3400340A148A100A118207CC
:10022000203449344D345034203400340A148A10B8
:100230000A118207533475346E3400340A148A105C
:100240000A1182074D346F346F346E3400340A144F
:100250008A100A118207543400340A148A100A11D1
:1002600082074D3400340A148A100A1182070C34B4
:1002700000340A148A100A11820746343134543487
:100280004534203452344F3454344F3452340034D3
:100290000A148A100A1182072A340034FE0A0C104C
:1002A0008A110A122B28070801397D060317C50099
:1002B00003130708FD000317451C6E290313470BA2
:1002C00067290130B0020030031C0130B102460B37
:1002D0006D290130B0070318B10A031703138C10FE
:1002E0008A110A122B288C1E73291808A8001A08D4
:1002F000F800A81C7D291812181600008A110A128D
:100300008229732978080317C70047081F3C031C7C
:100310008D2947080D3C031D94297608F60AA03E56
:10032000840083134708800003138C128A110A1279
:100330002B2824308400831700080319AC290630C9
:10034000F800F701F70BA229F80BA1297B30F70081
:10035000F70BA829800B9F29003403172B0EF039C7
:10036000F7000F300313060577048600000006141B
:100370000330F700F70BBA29061000348610F0306E
:100380008316860083120615000006140000060876
:10039000060E0F390317AB000313061000000614F6
:1003A000000000000000000000000608060E0F39E3
:1003B0000317AA0003130610003083168600831269
:1003C00003172B0EF700F030F70577082A04F80022
:1003D0007808AA00AA1FEE290313BF29A808031D45
:1003E000F52903138610F729031703138614000059
:1003F0000611000006100317290EAA000F30AA05E7
:100400002A08AB000313AD21031729080F39AA00EE
:10041000AB000313AD210034003083168600831235
:100420008610061106100F300317A400031399213C
:1004300001308316E1006108033C031C2D2A0330C0
:1004400083120317AB000313AD2105300317A4007B
:10045000031399218316E10A1B2A02308312031722
:10046000AB000313AD218316E1016108033C031CBB
:100470004C2A6108831247208316E2008312031777
:10048000A80183160313620883120317A90003133C
:10049000BE218316E10A352A83128A150A16F0282E
:1004A0000317250B542A572A4030A600582AA601C4
:1004B00001302402A60726088038A700A8012708D3
:1004C000A9000313BE21003403172308F7000C30E2
:1004D000770203130319752A0A3077020319812A58
:1004E000083077020319892A902A0317A8010130DE
:1004F000A9000313BE2102300317A400031399219E
:10050000982A01300317A4000230A50003135022DB
:10051000982A0317A8011030A9000313BE21982AB6
:1005200001300317A8002308A9000313BE21982A4D
:1005300000340B138B138B1B9A2A03173A08BB004A
:10054000BC018E0138088D003A088C0083168C138C
:100550000C15831203130B08F7008B138316031774
:1005600055308D00AA308D008C148C18B52A0C11D2
:100570007708831203138B04013003173807BB007D
:100580008E013B088D0039088C0083168C130C15E6
:10059000831203130B08F7008B13831603175530D0
:1005A0008D00AA308D008C148C18D42A0C11770879
:1005B000831203138B04C0308B04003464300317A0
:1005C00090009101A13092009301E13094009501D7
:1005D0002330960001309700643098000130990074
:1005E000A4309A0001309B00E3309C0001309D0054
:1005F00021309E0002309F005E30A0000230A1003A
:100600009A30A2000230A300D530A4000230A50029
:100610000F30A6000330A7004330A8000330A90024
:100620007530AA000330AB00A030AC000330AD0041
:10063000C930AE000330AF00EF30B0000330B1007E
:100640000D30B2000430B3001530B4000430B500F2
:100650008E0106308D0083168C130C1483120C0847
:10066000373C031D342B622B143083160313E10037
:10067000E2016208133C031C602B0310620D103E64
:1006800084008317840A0008E40084030008E30060
:10069000610883120317B8008316031364088312DA
:1006A0000317BA0083160313630883120317B900F4
:1006B0000313992202308316E1070130E207392B38
:1006C0008312031703138A150A160F298316E801EC
:1006D000E9016708831203178E0083160313660867
:1006E000831203178D0083168C130C1483120C08CD
:1006F00083160313E901E800053083120317A400F1
:100700000313992183166808EB00EA01013066079C
:10071000EC006708ED000318ED0A6D08831203175B
:100720008E00831603136C08831203178D00831643
:100730008C130C1483120C08831603136A04E8004C
:100740006B08E9006808F8006908F90083120034B2
:10075000F801F901F701FA0103172708031DB32B6C
:1007600026080319CD2B1030A8000310A40DA50DE9
:10077000F70DFA0D27087A02031DC02B2608770211
:10078000031CC92B2608F702031CFA032708FA02E8
:100790000314F80DF90DA80BB52B0000031300345A
:1007A00003171D08A5001C08A4000330A700E830AB
:1007B000A6000313A823780803179E001D08A500B0
:1007C0001C08A400A7016430A6000313A82379081D
:1007D0000317A3007808A2002308A5002208A4009C
:1007E000A7010A30A6000313A823770803179F0068
:1007F0001D08A5001C08A400A7010A30A6000313C9
:10080000A82379080317A3007808A2002308A500ED
:100810002208A400A7010A30A6000313A823770822
:100820000317A0001D08A5001C08A400A7010A309A
:10083000A6000313A82377080317A1009E08031935
:10084000292C30301E07A200A30003136422382C89
:100850000317A201220803134F2000380319382C74
:100860000317A20AA3000313642203172A2C0313FD
:1008700003179E08031D502C9F08031D502CA20136
:10088000220803134F20003803194E2C0317A20A25
:10089000A300031364220317402C0313562C0317E1
:1008A00030301F07A200A3000313642203179E0821
:1008B000031D712C9F08031D712CA008031D712CB2
:1008C000A201220803134F20003803196F2C0317CD
:1008D000A20AA300031364220317612C0313772CCD
:1008E000031730302007A200A30003136422303026
:1008F00003172107A200A3000313642200340B1383
:100900008B138B1B802C14308316E300E401E5016C
:100910006408123C031C1A2DE7016308E6008312E9
:10092000662379088316E2007808E100013083121B
:100930000317A400A500031350228316E6016608DE
:100940008312EB2000380319AF2C8316E60A8312BA
:100950000317A3000313642283169F2C8312013014
:100960000317A4000230A500031350228316E601EA
:1009700066088312052100380319C82C8316E60A7D
:1009800083120317A300031364228316B82C831267
:1009900003179D01831603136508831203179C0038
:1009A0000313D023DF300317A3000313642283163D
:1009B000E601660883120C2100380319E92C83161E
:1009C000E60A83120317A300031364228316D92CAB
:1009D000831283166208831203179D008316031384
:1009E0006108831203179C000313D0238316E016BB
:1009F0006008870000308312871A0130013C031D14
:100A0000072D01300317A40003139921F62C04309D
:100A10008316E600C83083120317A400031399213C
:100A20008316E60B0A2D0230E3076408E40A05305A
:100A3000E507882C83128A150A161F290B138B13BE
:100A40008B1B1F2DB1017C08B00001300317A400DF
:100A5000A500031350228316E40164088312A32027
:100A6000003803193D2D8316E40A83120317A300EF
:100A70000313642283162D2D831201300317A40063
:100A80000230A500031350228316E4016408831288
:100A9000BC2000380319562D8316E40A831203176D
:100AA000A300031364228316462D83128316851632
:100AB00000308312851A0130013C031D632D83161B
:100AC000E1018312562D04308316E400FA308312BC
:100AD0000317A400031399218316E40B662D01303C
:100AE00083120317A400A500031350228316E40108
:100AF00064088312BC2000380319882D8316E40A89
:100B000083120317A300031364228316782D831224
:100B1000C0308B0414308316E100E301E201E308E6
:100B2000031D512E62085A3C031C512EE01660082A
:100B3000870000308312871A0130013C031D2B2EE1
:100B400001300317A4000230A500031350228316BE
:100B5000E40164088312D52000380319B92D8316E7
:100B6000E40A83120317A300031364228316A92D3A
:100B7000831283166308831203179D0083160313E1
:100B80006208831203179C000313D0238316601599
:100B9000600887000030831207190130003A0319FA
:100BA000DC2D8316E014600887000030831287185C
:100BB0000130003A031D012E83166015600887007E
:100BC0000030831207190130003A031DEF2D013068
:100BD000C6008316E011600887008312871583160C
:100BE000E014600887000030831287180130003A53
:100BF000031D002E0130C700831605118312051551
:100C0000C62D83160511831205118316E0116008A5
:100C1000870083128711C601C7018316E4016408A7
:100C20008312DF20003803191F2E8316E40A831273
:100C30000317A3000313642283160F2E83123108B7
:100C400003179D000313300803179C000313D023E0
:100C50008316962D83120B138B138B1B2C2E0230B5
:100C60008316E400FA3083120317A40003139921BA
:100C70008316E40B322E610883120317B8000313A6
:100C800031080317BA00031330080317B900031320
:100C9000992202308316E1070530E2070318E30AC0
:100CA0008F2D023083120317B80003133108031786
:100CB000BA00031330080317B9000313992203176E
:100CC0008E0106308D0037308C0083168C130C1586
:100CD000831203130B08F7008B1383160317553089
:100CE0008D00AA308D008C148C18742E0C1177088E
:100CF000831203138B0404308316E400FA3083124A
:100D00000317A400031399218316E40B7E2E8A0196
:100D1000831200288A150A162F290B138B138B1B9D
:100D20008E2E01300317A400A50003135022831652
:100D3000E40164088312742000380319A92E831675
:100D4000E40A83120317A300031364228316992E67
:100D5000831201300317A4000230A50003135022B0
:100D60008316E40164088312892000380319C22E17
:100D70008316E40A83120317A30003136422831665
:100D8000B22E83128316E0166008870000308312AB
:100D9000871A0130013C031D0F2F83166015600870
:100DA00087000030831207190130003A0319E32E3F
:100DB0008316E01460088700003083128718013022
:100DC000003A031D042F8316601560088700003069
:100DD000831207190130003A031DF42E8316E01127
:100DE00060088700831287158316E0146008870067
:100DF0000030831287180130003A031D032F831639
:100E0000051183120515CD2E8316051183120511C8
:100E10008316E0116008870083128711C22E02300A
:100E20000317B800BA016430B900031399220430E3
:100E30008316E400FA3083120317A40003139921E8
:100E40008316E40B1A2F8A01831200288A150A16CA
:100E50003D291030F700FA010317B001AD0CAC0CBE
:100E6000031C382F2E08FA070318B00A2F08B00702
:100E7000B00CFA0CF90CF80CF70B2E2F03130034FE
:100E800020300317A1009D019E019F01A0011808B9
:100E9000FA001708F9001608F8001508F700031003
:100EA000771C602F19089D071A0803181A0F9E0750
:100EB0001B0803181B0F9F071C0803181C0FA00713
:100EC000A00C9F0C9E0C9D0CFA0CF90CF80CF70C66
:100ED000A10B4F2F03138A150A121C29F701F801E1
:100EE000F901FA010317AE01AF01B001B1012D08FC
:100EF0002C042B042A040319AD2F2030B200031058
:100F0000A60DA70DA80DA90DAE0DAF0DB00DB10D1D
:100F10002D083102031D962F2C083002031D962F39
:100F20002B082F02031D962F2A082E02031CA72F21
:100F30002A08AE022B08031C2B0FAF022C08031C3F
:100F40002C0FB0022D08031C2D0FB1020314F70D56
:100F5000F80DF90DFA0DB20B7F2F00002E30840032
:100F6000831703130034F701F80183166408031094
:100F70006518F707F70CF80CE518F707F70CF80CED
:100F80006519F707F70CF80CE519F707F70CF80CDB
:100F9000651AF707F70CF80CE51AF707F70CF80CC9
:100FA000651BF707F70CF80CE51BF707F70CF80CB7
:040FB0008312003474
:101000006F0803171602031C1228031D0D28031373
:101010006E0803171502031C12285A30F80000301E
:10102000F900E428980197019A0199019808031D95
:1010300057281708113C031C5728160803134B02A6
:10104000031C3228031D2C284A0803171502031C11
:101050002B280313322803130030F800F90003177C
:10106000E428031303100317170DF900180DFA00F5
:1010700079084A3E840083137A188317840A00088B
:10108000FA0084030008F80016087A02031C5328AB
:10109000031D4E2878081502031853281708031952
:1010A000980397035728970A0319980A162898084F
:1010B000031D5E281708113C03186228170803193E
:1010C00098039703013017079D0018089E00031826
:1010D0009E0A03101D0DF9001E0DFA0079084A3E04
:1010E000840083137A188317840A0008A0008403FD
:1010F00000089F000310170DF900180DFA00790879
:101100004A3E840083137A188317840A0008FA0081
:10111000840300081F02A1002008A2007A08031C13
:101120007A0FA2022208A5002108A400A701053019
:10113000A6008A110313A8238A15790803179C00B7
:1011400078089B001808AD001708AC00AF01053007
:10115000AE008A11031329278A15790803179E0008
:1011600078089D000310170DF900180DFA00790892
:101170004A3E840083137A188317840A0008FA0011
:101180008403000815029F001608A0007A08031CBB
:101190007A0FA0022008A5001F08A4001C08A700C1
:1011A0001B08A6008A110313A8238A1578080317C1
:1011B0001D0799001E089A0003189A0A79089A07D1
:1011C0001908F8001A08F900031300348430831654
:1011D0009F0083121F083839C1389F000830F8007B
:1011E0001F08C73978049F00A630F700F70BF628D0
:1011F00000001F151F19FA2883161E088312BA0053
:101200001E08BB00BC01BD013D0803179800031375
:101210003C080317970003133B08031796000313BA
:101220003A08031795009C019B0101309A00683031
:1012300099008A110313402F8A157A080317980022
:101240007908970078089600770895001808A90093
:101250001708A8001608A7001508A600AD01AC01E4
:101260000330AB009830AA008A1103136E278A1549
:101270007A08BD007908BC007808BB007708BA007E
:1012800005300317A4008A11031399218A151F083A
:1012900038399F00B4303A070317950003133B0811
:1012A00003179600003003180130960703133C081B
:1012B00003179700003003180130970703133D0808
:1012C0000317980000300318013098071808A90088
:1012D0001708A8001608A7001508A600AD01AC0164
:1012E0000130AB006830AA008A1103136E278A15FB
:1012F0000008BE00840A0008BF00840A0008C0007D
:10130000840A0008C100003403171608FA00150803
:10131000840083137A18831780080319D1291608CB
:101320009A001508990018089C0017089B001C08D3
:10133000FA001B08840083137A18831780080319A6
:10134000BC291A08FA001908840083137A18831735
:1013500000089D001C08FA001B08840083137A18FB
:10136000831700081D02031DBC29990A03199A0A54
:101370009B0A03199C0A97291C08FA001B08840081
:1013800083137A1883178008031DCB291508F800EA
:101390001608F900D429950A0319960A031384291B
:1013A00003170030F800F900031300340317AA01F3
:1013B000A8010A30A900A701A601240825040319E1
:1013C000EA292A08AA0A2407840083132518831708
:1013D0000008AB002B082D3C031DFA290130A800A2
:1013E0002A08AA0A240784008313251883170008F3
:1013F000AB00072A2B082B3C031D072A2A08AA0A40
:10140000240784008313251883170008AB002B08DA
:101410002F3C0318BE2A2B08393C031CBE2A2B087C
:10142000303C031D332A2A0824078400831325181F
:1014300083170008783C0319272A2A082407840008
:101440008313251883170008583C031D332A1030D6
:10145000A900AA0A2A08AA0A2407840083132518C7
:1014600083170008AB0029080A3C031D622A2B08D9
:101470002F3C0318612A2B08393C031C612AAD015B
:101480000A30AC002708AF002608AE008A1103130B
:1014900029278A1579080317AD007808AC00303089
:1014A0002B022C07A6002D08A7000318A70A2A085C
:1014B000AA0A240784008313251883170008AB00A9
:1014C000372ABE2A2908103C031DBE2A2B08603C7F
:1014D0000318712A2B087A3C031C712A2B08DF3968
:1014E000722A2B08AB002F3C03187A2A2B08393CB0
:1014F0000318822A2B08403C0318BE2A2B08463CBE
:10150000031CBE2A2B082F3C03189F2A2B08393CAA
:10151000031C9F2A260DAC00270DAD00AC0DAD0DB0
:10152000AC0DAD0DAC0DAD0DF030AC0530302B0277
:101530002C07A6002D08A7000318A70AB42A260D19
:10154000AC00270DAD00AC0DAD0DAC0DAD0DAC0D6F
:10155000AD0DF030AC0541302B020A3E2C07A60041
:101560002D08A7000318A70A2A08AA0A240784003E
:101570008313251883170008AB00662A29080A3C44
:10158000031DC92A280BC92AA609A709A60A0319F7
:10159000A70A2608F8002708F900031300340130D1
:1015A0000317A4001708A5008A11031350228A15F7
:1015B00003179C011C088A11031355208A15003853
:1015C0000319EC2A03179C0AA3008A11031364224F
:1015D0008A150317DA2A031303171B089D001A083C
:1015E0009C008A110313D0238A15DF300317A30050
:1015F0008A11031364228A1503179C011C088A119F
:1016000003135C208A1500380319102B03179C0A5A
:10161000A3008A11031364228A150317FE2A0313F9
:10162000031719089D0018089C008A110313D02382
:101630008A15DF300317A3008A11031364228A1569
:1016400012300317A4000130A5008A1103135022A1
:101650008A1503179C011C088A11031364208A153C
:10166000003803193D2B03179C0AA3008A110313AA
:1016700064228A1503172B2B031312300317A400BF
:101680000230A5008A11031350228A1503179C010A
:101690001C088A1103136C208A15003803195A2B71
:1016A00003179C0AA3008A11031364228A150317E7
:1016B000482B0313003401307602A03E84008313CC
:1016C00000080D3C031DA52E01307602A03E8400CB
:1016D00083138001031795019601E1308400831381
:1016E0001508840716088A11031355208A158000EF
:1016F00000380319802B0317960A950A6D2B0313E4
:10170000031795019601E5308400831315088407BB
:1017100016088A11031305218A1580000038031961
:10172000962B0317960A950A832B0313031795012B
:101730009601E930840083131508840716088A117E
:10174000031316218A15800000380319AC2B0317E8
:10175000960A950A992B03130317950196011030E9
:10176000840083171508840716088A1103131E21A5
:101770008A15800000380319C22B0317960A950AB0
:10178000AF2B031303179601A03095009801E130A9
:10179000970003138421780879040319F72B0317A2
:1017A0009601A03095009801E5309700031384213D
:1017B000780879040319F72B03179601A0309500D8
:1017C0009801E93097000313842178087904031DF8
:1017D0000B2C03179601A0309500013098001030B3
:1017E00097000313842178087904031D0B2C8316BA
:1017F00020084D3C031D022C7608053C031D022CDD
:1018000083120B2C2008573C031DA22E7608093C9E
:10181000031DA22E831203179701A001A10104301A
:10182000F8001830840083178001840AF80B142C08
:101830000430F8001C30840083178001840AF80B00
:101840001D2C95019601A301A030A2002308A5003C
:101850002208A4002508FA002408840083137A18BB
:10186000831780080319382CA40A0319A50A2A2C07
:1018700022082402F7002508FA002308031C230F7E
:10188000FA027708F8007A08F900F908031D4C2CD1
:10189000780815020318C42CA030150784008313A0
:1018A00000082E3C031D582CA0010130A100C22CC1
:1018B000A0301507840083130008203C031D632C0F
:1018C000A001A101C22CA0301507840083130008D9
:1018D0002F3C0318732CA0301507840083130008D5
:1018E000393C0318742CC22C210B772CC22CA00875
:1018F000031D7E2C9601970A0130A0001708F700FF
:1019000001307702031303198A2C0230770203197E
:10191000A52CC12C183003171607F8000130FA0067
:101920000318FA0A7808A2007A08A300A030150765
:10193000840083130008A400220884008313231862
:10194000831724088000960AC22C1C300317160740
:10195000F8000130FA000318FA0A7808A2007A08A1
:10196000A300A0301507840083130008A4002208F8
:10197000840083132318831724088000960AC22C3E
:1019800003130317950A232C0130A5001830A40077
:101990000313D62179080317A3007808A200A31B1C
:1019A000E92C0130A5001830A4000313D6217908D2
:1019B0000317A5007808A400A51BEC2C2508003C03
:1019C0000318EC2CFF3A031DE92C2408683C03188B
:1019D000EC2C0030F8006B2D0130A5001C30A40069
:1019E0000313D62179080317A3007808A200A31BCC
:1019F0000D2D0130A5001C30A4000313D621790859
:101A00000317A5007808A400A51B102DA508031D29
:101A10000D2D24085A3C0318102D0030F8006B2DB2
:101A20000130A5001830A4000313D6217808F70070
:101A30007908F800F901FA017A08C5007908C400AC
:101A40007808C3007708C200B43042070317A20029
:101A5000031343080317A300003003180130A30742
:101A6000031344080317A400003003180130A4072F
:101A7000031345080317A500003003180130A5071C
:101A80002508A9002408A8002308A7002208A6000A
:101A9000AD01AC010130AB006830AA008A1103131C
:101AA0006E278A150008B400840A0008B500840A6D
:101AB0000008B600840A0008B70001300317A5002B
:101AC0001C30A4000313D6217908B3007808B200B3
:101AD0000130F8000317F8080319A02E1030A400F5
:101AE0000130A5008A11031350228A1503179501AE
:101AF00015088A11031327218A15003803198A2D26
:101B00000317950AA3008A11031364228A15031789
:101B1000782D031343080317960003134208031795
:101B2000950001309700031333080317990003133E
:101B300032080317980016089B0015089A00031333
:101B4000CF22E62002303A07F7003B08F8000030C9
:101B500003180130F8073C08F90000300318013081
:101B6000F9073D08FA00003003180130FA077A0837
:101B70003702031CCD2D031D382E79083602031CB5
:101B8000CD2D031D382E78083502031CCD2D031DE5
:101B9000382E34087702031C382E0A303407031716
:101BA0009500031335080317960000300318013021
:101BB0009607031336080317970000300318013007
:101BC00097070313370803179800003003180130F4
:101BD00098070A3003133A070317990003133B08C9
:101BE00003179A000030031801309A0703133C08CA
:101BF00003179B000030031801309B0703133D08B7
:101C000003179C000030031801309C0702301902B2
:101C1000F7001A08F8000030031C0130F8021B0816
:101C2000F9000030031C0130F9021C08FA000030F2
:101C3000031C0130FA0218087A02031C4C2E031907
:101C4000232E0313382E17087902031C4C2E031978
:101C50002B2E0313382E16087802031C4C2E031962
:101C6000332E0313382E7708150203184C2E031356
:101C70000130F5003D088316DF0083123C0883160F
:101C8000DE0083123B088316DD0083123A088316B8
:101C9000DC004F2E83120317F50183160313831202
:101CA0003108031796000313300803179500031338
:101CB00000207908B9007808B80002303807F80029
:101CC0003908FA000318FA0A7A083302031C6E2E48
:101CD000031D9B2E32087802031C9B2E0A3032070C
:101CE0000317950003133308031796000318960A89
:101CF0000A30031338070317970003133908031733
:101D000098000318980A02301702F7001808FA0022
:101D10000030031C0130FA027708F80016087A0236
:101D2000031C9F2E0319962E03139B2E7808150271
:101D300003189F2E03130130F400A12E0317F401A2
:101D400003138316F601A00183128A150A16FA29D5
:1020000083166015600887000030831207190130BD
:10201000003A03192A288316E0146008870000306C
:10202000831287180130003A03192A2883160516EF
:1020300000308312051A0130003A03192A2883164A
:10204000E0166008870000308312871A0130003ADA
:10205000031D042C8316601560088700003083126E
:1020600007190130003A031940288316E01460086C
:1020700087000030831287180130003A031D722850
:102080008316E011600887008312871183160511FB
:102090008312051104308316E300FA30831203170C
:1020A000A4000A12031399210A168316E30B4D2884
:1020B0000230F4008312C601C701310803179600ED
:1020C00003133008031795000A128A150313002022
:1020D0000A168A117908B3007808B2003308B900EB
:1020E0003208B8008316051600308312051A013035
:1020F000003A031986288316E0166008870000302E
:102100008312871A0130003A031DB8288316601223
:1021100060088700831207128316851283128512C6
:1021200004308316E300FA3083120317A4000A1266
:10213000031399210A168316E30B93280230F50046
:102140008312C901C8010A128A15E6200A168A11EB
:102150003D08B7003C08B6003B08B5003A08B4009B
:102160004108C5004008C4003F08C3003E08C20043
:102170003F088316E40083123E088316E300023012
:1021800083120317970003133908031799000313E9
:102190003808031798008316031364088312031783
:1021A0009B00831603136308831203179A000A1215
:1021B0008A150313CF220A168A1143088316E400F6
:1021C000831242088316E30001308312031797003D
:1021D00003133308031799000313320803179800F9
:1021E000831603136408831203179B0083160313DB
:1021F0006308831203179A000A128A150313CF2269
:102200000A168A1183160C14FE017E080B3C031C6F
:10221000752B0130E100E830E200601560088700AE
:102220000030831207190130003A031D7C29831600
:10223000E014600887000030831287180130013CE9
:10224000031D7C29B308031D2D293208593C031CAA
:102250002D290130B2070318B30A831662088312CE
:102260000317A4000A12031399210A1683166108A2
:10227000E10AE1006208133C031852290A30E40025
:102280006108E5000A128312B3270A16780883163C
:10229000E4006108E5000A128312B3270A167808E1
:1022A0008316E202831243088316E4008312420875
:1022B0008316E300013083120317970003133308DA
:1022C00003179900031332080317980083160313AA
:1022D0006408831203179B00831603136308831299
:1022E00003179A000A128A150313CF220A168A11BD
:1022F000FE0183160D2983128316E01460088700FF
:102300000030831287180130003A031DEB29831631
:102310006015600887000030831207190130013C06
:10232000031DEB29B208031D9829B30803199E2940
:102330000130B2020030031C0130B3028316620880
:1023400083120317A4000A12031399210A16831695
:102350006108E10AE1006208133C0318C3290A304E
:10236000E4006108E5000A128312B3270A16780810
:102370008316E4006108E5000A128312B3270A16E7
:1023800078088316E202831243088316E40083125E
:1023900042088316E30001308312031797000313EA
:1023A00033080317990003133208031798008316A4
:1023B00003136408831203179B0083160313630837
:1023C000831203179A000A128A150313CF220A16E2
:1023D0008A11FE017C298316E01660088700003010
:1023E0008312871A0130003A031DB12A831605169D
:1023F00000308312051A0130013C031DB12AB708D1
:10240000031D1D2AB608031D1D2A3508013C031CA7
:102410001D2A031D0F2A3408673C031C1D2A0130A6
:10242000B407003003180130B5070030031801303D
:10243000B607003003180130B7078316620883120D
:102440000317A4000A12031399210A1683166108C0
:10245000E10AE1006208133C0318422A0A30E40052
:102460006108E5000A128312B3270A16780883165A
:10247000E4006108E5000A128312B3270A167808FF
:102480008316E202B430831234078316E30083120A
:1024900035088316E400003003180130E407831286
:1024A00036088316E500003003180130E507831273
:1024B00037088316E600003003180130E607660887
:1024C00083120317A90083160313650883120317E9
:1024D000A80083160313640883120317A70083164A
:1024E0000313630883120317A600AD01AC0101308A
:1024F000AB006830AA000A1203136E270A16000800
:10250000C200840A0008C300840A0008C400840AC8
:102510000008C50043088316E400831242088316AE
:10252000E3000130831203179700031333080317E6
:1025300099000313320803179800831603136408E5
:10254000831203179B008316031363088312031778
:102550009A000A128A150313CF220A168A11FE0165
:10256000EB298316051600308312051A0130003A54
:10257000031D732B8316E01660088700003083125A
:10258000871A0130013C031D732BB408031DD12AA7
:10259000B508031DD12AB608031DD12AB7080319AF
:1025A000DF2A0130B4020030031C0130B5020030D4
:1025B000031C0130B6020030031C0130B702831641
:1025C000620883120317A4000A12031399210A1642
:1025D00083166108E10AE1006208133C0318042B2A
:1025E0000A30E4006108E5000A128312B3270A16D4
:1025F00078088316E4006108E5000A128312B32705
:102600000A1678088316E202B43083123407831660
:10261000E300831235088316E4000030031801300C
:10262000E407831236088316E500003003180130F2
:10263000E507831237088316E600003003180130DF
:10264000E607660883120317A900831603136508BB
:1026500083120317A8008316031364088312031759
:10266000A70083160313630883120317A600AD01A6
:10267000AC010130AB006830AA000A1203136E27C8
:102680000A160008C200840A0008C300840A000871
:10269000C400840A0008C50043088316E4008312BE
:1026A00042088316E30001308312031797000313D7
:1026B0003308031799000313320803179800831691
:1026C00003136408831203179B0083160313630824
:1026D000831203179A000A128A150313CF220A16CF
:1026E0008A11FE01B12A831605290C1010308312BD
:1026F0000317A4000130A5000A12031350220A1682
:102700008316E30163080A1283122D210A1600388A
:102710000319962B8316E30A83120317A3000A12E8
:10272000031364220A168316822B831231080317BF
:10273000960003133008031795000A128A15031335
:1027400000200A168A117908B9007808B8003908FB
:102750003302031CB12B031DBB2B32083802031CB0
:10276000BB2B33083902031CBE2B031DBB2B3808BF
:1027700032020318BE2B0130F400BF2BF4010A1201
:102780008A15E6200A168A113D083702031CDA2B47
:10279000031DF02B3C083602031CDA2B031DF02B23
:1027A0003B083502031CDA2B031DF02B34083A02D8
:1027B000031CF02B37083D02031C032C031DF02BD8
:1027C00036083C02031C032C031DF02B35083B028A
:1027D000031C032C031DF02B3A0834020318032CAE
:1027E0000130F5003D088316DF0083123C08831694
:1027F000DE0083123B088316DD0083123A0883163D
:10280000DC00052C8312F501831683128A150A1643
:02281000FD29A0
:10300000840183131F308305063083169F008312CB
:10301000A801FF3083169900223098009030831267
:103020009800A901AA010130AB00AC01AD01AE01CD
:103030000230AF00B001B101B201B301B401B5017A
:10304000B601B701B801B901BA01BB01BC01BD01AC
:10305000BE01BF01C001C101C201C301C401C5015C
:10306000C601C701C801C901CA01CB01CC01CD010C
:10307000CE01CF01D001D101D201D301D401D501BC
:10308000D601D701D801D901DA01DB01DC01DD016C
:10309000DE01DF01E001E101E201E301E401E5011C
:1030A000E601E701E801E901EA01EB01EC01ED01CC
:1030B000EE01EF018316A001A101A201A301A40169
:1030C000A501A601A701A801A901AA01AB01AC01B4
:1030D000AD01AE01AF01B001B101B201B301B40164
:1030E000B501B601B701B801B901BA01BB01BC0114
:1030F000BD01BE01BF01C001C101C201C301C401C4
:10310000C501C601C701C801C901CA01CB01CC0173
:10311000CD01CE01CF01D001D101D201D301D40123
:10312000D501D601D701D801D901DA01DB01F001BF
:10313000F101F201F301F401F501F6016430FC0044
:10314000FD01FE01DC01DD01DE01DF01FF30E000F9
:10315000F701F71DB6280730831281018130840002
:1031600083130008C0390F38800083166400813053
:1031700084000008C03977048000B53083129000C5
:103180007830F80006389200C530831692000C1093
:103190008C1483121F0838399F0083168C16C03098
:1031A00083128B0413308316850000308600E730CD
:1031B0008700E000E0116008870083128711831602
:1031C00005118312051183166012600887008312AF
:1031D000071283168512831285120A128A110C2A8D
:1031E0000A168A158316E10161080A128A118312F0
:1031F00033210A168A15003803190C298316E10AAF
:1032000083120317A3000A128A11031364220A16F9
:103210008A158316F42883120A128A11DE2A0A16E6
:103220008A1583166015600887000030831207191D
:103230000130003A031D21290A128A117F2C0A1637
:103240008A158316E01460088700003083128718FF
:103250000130003A031D31290A128A111E2D0A1667
:103260008A158316051600308312051A0130003ABC
:10327000031D3F290A128A118D2E0A168A158316FC
:10328000E7010230E6000A128A11831266230A1649
:103290008A157908B1007808B0001430F000F10107
:1032A0007108123C031C76290310710D4A3E8316E7
:1032B000E100E2010318E20AE7017008E6000A12E1
:1032C0008A11831266230A168A1583166108840000
:1032D000831362188317840A7908800084037808AE
:1032E00080000230F007F10A8312502931080317D9
:1032F000960003133008031795000A1203130020E9
:103300000A167908B9007808B8003908B3003808F7
:10331000B2000A12E6200A163D08B7003C08B600C3
:103320003B08B5003A08B4008316E10161080A12AF
:103330008A11831233210A168A1500380319AE291F
:103340008316E10A83120317A3000A128A110313DA
:1033500064220A168A1583169629831205300317EC
:10336000A4000130A5000A128A11031350220A1684
:103370008A158316E10161080A128A118312392124
:103380000A168A1500380319D3298316E10A831215
:103390000317A3000A128A11031364220A168A155E
:1033A0008316BB29831210300317A4000230A50036
:1033B0000A128A11031350220A168A158316E10194
:1033C00061080A128A11831248210A168A150038E8
:1033D0000319F8298316E10A83120317A3000A12BE
:1033E0008A11031364220A168A158316E0298312B0
:1033F0000A125B2B0A168A1100288A150A12E62087
:103400000A16740BF72B10300317A4000230A50026
:103410000A128A11031350220A168A158316E10133
:1034200061080A128A1183124F200A168A15003881
:103430000319282A8316E10A83120317A3000A122C
:103440008A11031364220A168A158316102A83121E
:1034500083168C1283123108031796000313300869
:10346000031795000A12031300200A167908B90001
:103470007808B80033088316E200831232088316F6
:10348000E100620883120317A50083160313610885
:1034900083120317A400A7010530A6000A128A119F
:1034A0000313A8230A168A1579088316E4007808FE
:1034B000E300640883120317AD0083160313630847
:1034C00083120317AC00AF010530AE000A128A1157
:1034D000031329270A168A15780883166102E50066
:1034E0006208E6007908031C790FE60201306307E1
:1034F00083120317900083160313640883120317C3
:1035000091000318910A0310100DF900110DFA0033
:1035100079084A3E840083137A188317840A0008C6
:103520009300840300089200031083160313630DB5
:10353000F900640DFA0079084A3E840083137A1872
:103540008317840A0008FA00840300088312031713
:1035500012029400130895007A08031C7A0F950252
:103560001508A5001408A400A7010530A6000A123A
:103570008A110313A8230A168A1579088316EA000C
:103580007808E9000310630DF900640DFA0079086A
:103590004A3E840083137A188317840A0008831232
:1035A0000317910084030008900083160313660834
:1035B00083120317AD0083160313650883120317E4
:1035C000AC00831603136A0883120317AF00831637
:1035D0000313690883120317AE000A128A1103133A
:1035E00029270A168A15780803171007831603136C
:1035F000E70083120317110883160313E80003186A
:10360000E80A7908E8076708F8006808F900790807
:10361000F3007808F2008312C7080319552B31080C
:103620007302031C552B031D192B30087202031C57
:10363000552B83160511831205113F088316E200EE
:1036400083123E088316E1000230831203179700AD
:103650000313390803179900031338080317980058
:10366000831603136208831203179B008316031348
:103670006108831203179A000A120313CF220A1655
:103680000230F40006308316E100FA30831203178B
:10369000A4000A128A11031399210A168A158316A7
:1036A000E10B452B8312C701F72BC6080319A02B8A
:1036B00073083102031CA02B031D622B7208300219
:1036C000031CA02B8316E01160088700831287116A
:1036D0003F088316E20083123E088316E1000230A1
:1036E0008312031797000313390803179900031374
:1036F0003808031798008316031362088312031710
:103700009B00831603136108831203179A000A12A1
:103710000313CF220A160230F40006308316E100AC
:10372000FA3083120317A4000A128A110313992195
:103730000A168A158316E10B902B8312C601F72B0C
:1037400073083102031CCC2B031DAA2B3008720214
:103750000318CC2BC6080319C52B8316E01160088B
:1037600087008312871106308316E100FA30831236
:103770000317A4000A128A11031399210A168A1545
:103780008316E10BB62B8312C6010130C7008316E6
:10379000051183120515F72B31087302031CF72B53
:1037A000031DD62B720830020318F72BC708031924
:1037B000EF2B831605118312051106308316E100E5
:1037C000FA3083120317A4000A128A1103139921F5
:1037D0000A168A158316E10BE02B8312C70101300C
:1037E000C6008316E0116008870083128715750BE9
:1037F000DE2D10300317A4000230A5000A128A1132
:10380000031350220A168A158316E10161080A1271
:103810008A1183124F200A168A15003803191E2CAC
:103820008316E10A83120317A3000A128A110313F5
:1038300064220A168A158316062C831283168C12AC
:103840000A128312E6200A163D083702031C5B2C7D
:10385000031D3A2C3C083602031C5B2C031D3A2C3A
:103860003B083502031C5B2C031D3A2C34083A023A
:1038700003185B2C3A0834028316E30083123508E0
:103880008316E40083123B08031C3B0F482C4B2C8F
:103890008316E402831283165C0883123A028316AD
:1038A000E10083123B088316E2005D08031C5D0FF4
:1038B000E2027C2C831234083A028316E30083125E
:1038C0003B088316E40083123508031C350F692C6E
:1038D0006C2C8316E40283123A0883165C02E10022
:1038E0005D08E20083123B08031C3B0F782C7B2C05
:1038F0008316E202831283168312C9080319D22C9D
:1039000037083D02031CD22C031D962C36083C02BE
:10391000031CD22C031D962C35083B02031CD22C11
:10392000031D962C34083A02031CD22C83168512F0
:10393000831285123F088316E60083123E08831621
:10394000E5000230831203179700031339080317A9
:1039500099000313380803179800831603136608A9
:10396000831203179B008316031365088312031742
:103970009A000A120313CF220A1606308316E500B6
:10398000FA3083120317A4000A128A110313992133
:103990000A168A158316E50BC02C0230F500831237
:1039A000C901DE2DC8080319292D3D083702031C63
:1039B000292D031DEB2C3C083602031C292D031D69
:1039C000EB2C3B083502031C292D031DEB2C3A0878
:1039D0003402031C292D83166012600887008312AD
:1039E00007123F088316E60083123E088316E5009F
:1039F0000230831203179700031339080317990045
:103A000003133808031798008316031366088312FC
:103A100003179B00831603136508831203179A008C
:103A20000A120313CF220A1606308316E500FA3075
:103A300083120317A4000A128A11031399210A168C
:103A40008A158316E50B172D0230F5008312C80185
:103A5000DE2D37083D02031C862D031D3F2D360841
:103A60003C02031C862D031D3F2D35083B02031C21
:103A7000862D031D3F2D3A0834020318862DC908F0
:103A80000319582D8316851283128512063083166A
:103A9000E500FA3083120317A4000A128A110313F7
:103AA00099210A168A158316E50B492D8312C9013F
:103AB0000130C80083166012600887008312071661
:103AC0008316E408031D682D6308073C03186F2D57
:103AD000E208031D842D6108073C031C842D83121A
:103AE00007128316601260088700053083120317DF
:103AF000A4000A128A11031399210A168A150716BF
:103B000083166012600887008312DE2D3D0837029D
:103B1000031CDE2D031D9C2D3C083602031CDE2DEC
:103B2000031D9C2D3B083502031CDE2D031D9C2D1F
:103B300034083A020318DE2DC8080319B72D83167E
:103B40006012600887008312071206308316E500B2
:103B5000FA3083120317A4000A128A110313992161
:103B60000A168A158316E50BA82D8312C8010130A9
:103B7000C90083168512831285168316E408031D77
:103B8000C52D6308073C0318CC2DE208031DDD2D6D
:103B90006108073C031CDD2D8312851283168512F4
:103BA000053083120317A4000A128A110313992106
:103BB0000A168A15851683168512831275087404F1
:103BC000023C031D232E7408023C031DF82D023015
:103BD0000317B800031331080317BA0003133008A2
:103BE0000317B9000A128A11031399220A168A15BB
:103BF000F601F501F40183168C16103083120317B9
:103C0000A4000230A5000A128A11031350220A16DA
:103C10008A158316E10161080A128A11831248216C
:103C20000A168A1500380319232E8316E10A831217
:103C30000317A3000A128A11031364220A168A15B5
:103C400083160B2E83123F088316E20083123E0870
:103C50008316E1000230831203179700031339081B
:103C600003179900031338080317980083160313EA
:103C70006208831203179B008316031361088312E3
:103C800003179A000A120313CF220A16F8296300B9
:02400E00323F3F
:00000001FF
